:0400000045EF05F0D3
:10000800D9CF19F0DACF1AF0E1CF17F0E2CF18F014
:10001800E9CF15F0EACF16F02CEC05F0000015C07A
:10002800E9FF16C0EAFF17C0E1FF18C0E2FF19C0D8
:08003800D9FF1AC0DAFF110024
:100040000401376B1E0E716E0401400E096F5B0ECA
:100050000A6F040E0B6F880E086F9B0E0E6F040E56
:0A0060000F6F0D6B400E0C6F1200C5
:10006A0004012A6B14EE9BF024EE18F0010E2A5DAF
:10007A0004E2E6CFDEFF2A2BF9D7010E3E6F3F6B73
:02008A00120062
:10008C0004012A6B14EE20F024EE18F0020E2A5D07
:10009C0004E2E6CFDEFF2A2BF9D7020E3E6F3F6B50
:0200AC00120040
:1000AE000401010E135D04E0030E135D0EE016D085
:1000BE00000E125D04E0010E125D06E00FD0020E7E
:1000CE00396F35EC00F00AD009D0000E125D01E058
:1000DE0005D0020E396F46EC00F000D0180E3A6FC4
:0800EE00040E3B6F3493120075
:1000F6000401020E135D04E0030E135D0CE016D03E
:10010600000E125D01E012D0020E396F5B0E3C6FDD
:10011600040E3D6F0BD0000E125D01E007D0020EFB
:0E012600396F200E3C6F040E3D6F00D01200AA
:100134000401010E396F716A726A736A746A756AAE
:10014400766A776A786A796A7A6A7B6A7C6A7D6A8F
:100154007E6A7F6A326B336B12C431F4125103E14D
:10016400050E306F04D0060E306F20EC00F0120044
:100174000401800E10634FD0135103082FE0135174
:1001840002080EE01351010801E044D0010E396F5A
:10019400E20E3A6F0A0E3B6F120E3E6F3F6B3AD07F
:1001A400010E396F450EE16E040EE26E1245E12632
:1001B400000EE222E6CF3AF4E7CF3BF4F86AF76A9E
:1001C400040E3A25F66E3B51F7220900F5CF3EF4B2
:1001D40009000A00F5CF3FF40A001CD0010E396F64
:1001E400020E126502D0030E126F490EE16E040E68
:1001F400E26E1245E126000EE222E6CF3AF4E7CFA2
:100204003BF43AC4F6FF3BC4F7FF0800F5503E6FD9
:080214003F6B00D0348312009F
:10021C000401010E125D0CE110511F0B000808E1E6
:10022C00010E396F030E115D02E1348101D034915E
:10023C00000E125D37E110511F0B020833E114510F
:10024C000F0B00082FE0010E396F14510F0B080D26
:10025C00F350296B000F286F040E29231451800BC7
:10026C0001E0010E040DF35028253C6F000E2921EE
:10027C003D6F030E115D07E1840E3CC4E1FF3DC4EC
:10028C00E2FFE76E0FD014AF07D0000E3CC4E1FFC5
:10029C003DC4E2FFE76E06D0880E3CC4E1FF3DC4CE
:0602AC00E2FFE76E120004
:1002B2000401186B196B10511F0B020812E0105148
:1002C2001F0B01080BE010511F0B000801E029D0A1
:1002D200010E396F34A101D0188323D0010E396F7A
:1002E20020D0010E396F14510F0B080DF350296BFA
:1002F200000F286F040E29231451800B01E0010E18
:10030200040DF35028253C6F000E29213D6F3CC49B
:10031200E1FF3DC4E2FFE750040B02E0010E186F5B
:1003220000D0010E396309E1180E3A6F040E3B6FDB
:0C0332003493020E3E6F3F6B00D01200AF
:10033E000401080E3E5D000E3F5905E23EC440F436
:10034E003FC441F404D0080E406F000E416F049379
:10035E0004914151030B041340C405F440513E5F18
:10036E0041513F5B180E3C6F040E3D6F34A319D004
:10037E003AC4F6FF3BC4F7FFF86A3CC4E1FF3DC444
:10038E00E2FF4051411105E1F6CF3AF4F7CF3BF4CD
:10039E001ED00900F5CFE6FF0900400701E2410734
:1003AE00F0D73AC4E1FF3BC4E2FF3CC4D9FF3DC4E1
:1003BE00DAFF4051411105E1E1CF3AF4E2CF3BF4CF
:1003CE0006D0E6CFDEFF400701E24107F2D712006A
:1003DE000401020E135D04E0030E135D15E01CD044
:1003EE00000E125D01E018D02A6B14EE5BF024EEC5
:1003FE009BF0010E2A5D04E2E6CFDEFF2A2BF9D731
:10040E00010E3E6F3F6B08D0000E125D01E004D06E
:0A041E00020E3E6F3F6B00D012008B
:100428000401000E386F080E016F100E026F040EE3
:0C043800036F880E006F000E046F1200AE
:1004440004011051600BE842E842E842E842E84205
:10045400000858E111510C0854E01151070851E00B
:1004640011510B0843E011510A0832E011510308FD
:100474002CE01151010829E01151000823E0115129
:10048400080815E0115109080FE01151060809E0A8
:100494001151050801E036D0010E396F040E306F9A
:1004A40031D0BAEC00F02ED09AEC00F02BD0010E33
:1004B400396F310E3A6F040E3A6F3493010E3E6F6A
:1004C4003F6B20D059EC01F01DD00EEC01F01AD096
:1004D400010E396F14513A6F3B6B320E3A27040EFA
:1004E4003B233493010E3E6F3F6B0CD0010E396FEA
:1004F400E26A320E1425E16E040EE22212C4E7FF12
:0605040001D000D012003E
:10050A00040110511F0B010870E1145100086DE13C
:10051A001151060801E027D01351210807E01351B1
:10052A00220811E0135123081BE01BD0020E396F79
:10053A00010E316304D02A0E3A6F0B0E3B6F090E7F
:10054A003E6F3F6B0ED0020E396F010E316307D03A
:10055A00580E3A6F0B0E3B6F2F0E3E6F3F6B01D05A
:10056A0000D0348300D01051600BE842E842E842E0
:10057A00E842E842010839E111510B0831E0115112
:10058A00030823E011510A081BE0115102080DE08B
:10059A001151090807E01151010801E026D057EC72
:1005AA0000F023D07BEC00F020D0020E396F350E1C
:1005BA003A6F040E3B6F3493010E3E6F3F6B15D0BA
:1005CA00020E396F1351356F10D0020E396F360E85
:1005DA003A6F040E3B6F3493010E3E6F3F6B05D0AA
:0C05EA00020E396F1251366F00D0120063
:1005F6000401000E39630AD0080E016F100E026F57
:10060600040E036F840E006F046F2CD010AF1CD045
:100616003E51165D3F51175904E216C43EF417C405
:100626003FF49FEC01F0010E386F080E016F100EBB
:10063600026F040E036F800E006F180E066F040E15
:10064600076FC80E046F0ED0020E386F056BC80E0A
:10065600046F080E016F180E026F040E036FC80EAA
:0A066600006F00D06D9800D0120064
:100670000401030E0015436F01C442F442513E27AA
:1006800043513F23180E3A6F040E3B6F3AC4E1FF0B
:100690003BC4E2FF3CC4D9FF3DC4DAFF42514311E1
:1006A00005E1E1CF3AF4E2CF3BF406D0E6CFDEFF3E
:0A06B000420701E24307F2D71200EF
:1006BA000401376B08BF1BD009512C6502D009C44D
:1006CA002CF4376B14EE5BF02DC4D9FF2EC4DAFF7D
:1006DA002C51375D04E2E6CFDEFF372BF9D7400E07
:1006EA00096F400E0817087D880E081300D037518D
:0206FA001200EC
:1006FC000401040E306309D012C46EFF6E5003E087
:10070C00050E306F02D0030E306F010E38630AD025
:10071C009FEC01F004BD03D0C80E046F02D0880E0C
:0C072C00046F03D014EC02F000D01200A7
:100738000401020E38630FD038EC03F0020E39635F
:1007480002D0EFEC01F000BD03D0C80E006F02D05C
:0E075800880E006F03D014EC02F000D01200E7
:100766000401000E386F000E396F3E6B3F6B22ECB2
:1007760002F0000E396302D085EC02F0FBEC02F0C9
:0207860012005F
:1007880004016A6A686A9F0E6B6E3B0E696E6E6A38
:10079800716A726A736A746A756A766A776A786A5D
:1007A800796A7A6A7B6A7C6A7D6A7E6A7F6A160ED3
:1007B800706E68A602D06896FCD76D9814EC02F0AB
:0A07C8003491316B030E306F120004
:0A07D2000401698468986D8212002A
:1007DC009C0E0C6ED70E0D6E0D2EFED70C2EFCD76C
:0207EC001200F9
:0A07EE0004016D92699468941200F2
:0607F8000401689C1200E0
:1007FE0004017C0E6C142F6F000E2F6302D00FEFCE
:10080E0004F0040E2F6302D01BEF04F01EEF04F071
:10081E0000513C0BE842E8420D0803E1B3EC03F053
:10082E0002D09CEC03F003D07EEC03F000D012005B
:10083E0004017C0E6C142F6F080E2F6302D02FEF65
:10084E0004F00C0E2F6302D039EF04F03AEF04F0EF
:10085E0057C42DF458C42EF4010E2C6F5DEC03F02A
:08086E00446F01D000D012001C
:10087600040170A003D014EC02F07090689A120084
:060886000401689212005B
:10088C003D0E0B6EE10E0C6E3F0E0D6E0D2EFED757
:0E089C000C2EFCD70B2EFAD700000000120025
:1008AA0004016DB61200140E6F6E000E306F346BB9
:1008BA00316B6D6A696A6D86010E306FEEEC03F07A
:1008CA006DBA06D0686A696A69806988020E306FF3
:0208DA0012000A
:1008DC0004010CBFFED7400E2C6502D0400E2C6FCD
:1008EC002A6B2DC4E1FF2EC4E2FF24EE9BF02C51A9
:1008FC002A5D04E2E6CFDEFF2A2BF9D704012CC4D3
:0E090C000DF4400E0C170C7D880E0C1312001B
:10091A00E9CF51F4EACF52F4E1CF53F4E2CF54F4E1
:10092A00D9CF55F4DACF56F40401000E306301D062
:10093A0033D069A404D068A402D0F7EC03F06DB2F6
:10094A002BD069A004D068A002D0C4EC03F069A837
:10095A0004D068A802D0E9EC03F069AC04D068AC12
:10096A0002D0FCEC03F069AA04D068AA02D03BECDE
:10097A0004F069A204D068A202D043EC04F0030E8A
:10098A00306101D009D069A607D068A605D0FFEC6E
:10099A0003F01FEC04F0689656C4DAFF55C4D9FF79
:1009AA0054C4E2FF53C4E1FF52C4EAFF51C4E9FF51
:0209BA00120029
:1009BC00E0CF14F004EE00F0050EEE6AEA62FDD70B
:1009CC0046EC04F00401060E456F0B0E466F060E46
:1009DC00476F0B0E486F1A0E496F0C0E4A6FEA0EDA
:1009EC004B6F0B0E4C6FB60E4D6F0B0E4E6F220EE7
:1009FC004F6F0C0E506F1EC057F41FC058F420C020
:100A0C0059F421C05AF455EC04F0A19AA08AF28C46
:080A1C00F28E1450E06E12008E
:100A2400F26AF50EF16EC00EF06ED09E9D6AA06A59
:100A34009E6AA16A0F0EC112926A936AFF0E946EA7
:100A4400FF0E956E070E966E896A8A6A8B6A8C6AA7
:040A54008D6A120095
:100A5800A0AA05D0A1AA03D08DEC04F0A19A120097
:100A680004010CAF02D0006A1200A09A1EC02DF437
:100A78001FC02EF420C02CF42DDFA08A010E006EBA
:020A880012005A
:100A8A00CCDF1C0E1E6E000E1F6E1B0E206E000E9B
:100A9A00216E8FDF1D6AFF0E1D5C1CE21DC01BF05C
:100AAA001B0E1E6E000E1F6E010E206ED8DF005246
:100ABA0001E1F6D73D0E0B6EE10E0C6E3F0E0D6E88
:100ACA000D2EFED70C2EFCD70B2EFAD700000000F5
:080ADA001D2AE1D7DFD7FFD789
:100AE20012000100000002000000000000000800E7
:100AF20034001200010000000100000001000200A9
:100B020000000100090002002900000001000100AC
:100B12000000A000320009000400000000000200F2
:100B22000300000000000000090021000100010094
:100B32000000010022002F000000070005008100D4
:100B4200030040000000010007000500010003004F
:100B52004000000001000600A000FF0009000100A3
:100B6200A10001000900030015000000260000009A
:100B7200FF007500080095000100810002000900D5
:100B820004001500000026000000FF0075000800A8
:100B92009500010091000200090005001500000007
:100BA20026000000FF007500080095000200B10059
:040BB2000200C0007D
:100BB6001A00030050000000720000006F000000E1
:100BC600640000007500000063000000740000006F
:100BD6002D0000004E000000610000006D000000C6
:040BE60065000000A6
:100BEA001800030056000000650000006E000000B7
:100BFA00640000006F000000720000002D00000079
:100C0A004E000000610000006D0000006500000059
:080C1A000400030009000400BE
:040C220002000300C9
:020000040030CA
:0E000000200E211EFF0080FF0340036003401E
:00000001FF
